:020000040000FA
:06000000023003303A2833
:08000800A000030EA100831209
:1000100005191128831601178312B2308100B1012E
:100020002C2883160113831203140B190310A80D37
:10003000A90DAA0DAB0DAC0DAC16FF302C02031DA3
:100040002C28FA302B02031D2C2832152A08AF0069
:100050002908AE002808AD008B100B11210E83007B
:06006000A00E200E0900B5
:04006600003400342E
:0C007400203084008001840A6030040207
:10008000031C3C2862218316FF23900083128316F1
:100090000C3085058701831285018701073099009F
:1000A0000030831691009F008312C83083168100B0
:1000B000831231309000003083168C008312103090
:1000C0008B009A2181018E018F010B118B100B1077
:1000D0008C018B17792032198520B40B77280310F7
:1000E00085190314BA0DF0303A020319E2209B215E
:1000F0006A2864003310B10A311F8428AC01AB01B7
:10010000AA01A901A801B101080032110130B7000C
:100110008B132030370783169B001C141A08831298
:10012000A4001030370783169B001C141A08831292
:10013000A300A6000230A6060030370783169B00F6
:100140001C141A088312A200A7000130A7068B17FF
:10015000331CB02822090339A200A309A409A50968
:1001600024082F02031DDC2823082E02031DC328A8
:1001700022082D02031DDC2801303702031DC3288D
:100180003E143F14772126082E02031DD32827088A
:100190002D02031DDC2801303702031DD2283E103A
:1001A0003F148121DC285F08F039A03C0319DC28CA
:1001B0002E1ADC28DB288B21B70A023037020318FD
:1001C000080088280130B600B400B500B7008501EA
:1001D0008701B21395213D217920B40B0A29031020
:1001E00085190314BA0DF0303A02031932290C1C98
:1001F00006290C10C00A4108400203190429410ACB
:10020000400203193D21062985018701B50B0A2902
:10021000FA30B500321DEC283211331C14292D0997
:100220000339AD00AE09AF092F1CEC282D083002B0
:100230000319EC282D08B0002E1EEC288B1320305B
:100240003707BC002F08BB004F2110303707BC0018
:100250002E08BB004F2100303707BC002D08BB0023
:100260004F218B17850187019921B70AB60102300A
:100270003702031CEC289A2108008E018F01C0016F
:100280000C10013037020319902108003F1C0800B0
:100290003F101030BC003E08BB004F2108008B13FC
:1002A0003B0883161C159A003C089B0055309D00A6
:1002B000AA309D009C1464009C185B291C118312B9
:1002C0008B170800831600309B001C141A08831239
:1002D000DF00831620309B001C141A088312C10013
:1002E0000130C11BC100C1080319C10008008512FB
:1002F0000512851405148E018F010C104108C000F1
:10030000080085100510851605168E018F010C104A
:100310004108C0000800851005108512051208006C
:10032000380933398500B8000800B801B81438140A
:100330000800080008005F080F390A3C0319A829C3
:100340000C1C08000C10C00B08004108C0008501FF
:020350000800A3
:084000000100030006000900A5
:02400E00CC01E3
:10420000010078007A007C007E007B0079007F004E
:104210007D007A0078007E007C00FF00FF00FF0038
:104220000000F200F600FA00FE00F200F600FA00CC
:10423000FE00F200F600FA00FE00FF00FF00FF00A3
:10424000010005000500050005000900090009003E
:1042500009000D000D000D000D00FF00FF00FF0024
:10426000FF00FF00FF00FF00FF00FF00FF00FF0056
:10427000FF00FF00FF00FF00FF00FF00FF00FF0046
:10428000FF00FF00FF00FF00FF00FF00FF00FF0036
:10429000FF00FF00FF00FF00FF00FF00FF00FF0026
:1042A000FF00FF00FF00FF00FF00FF00FF00FF0016
:1042B000FF00FF00FF00FF00FF00FF00FF00FF0006
:1042C000FF00FF00FF00FF00FF00FF00FF00FF00F6
:1042D000FF00FF00FF00FF00FF00FF00FF00FF00E6
:1042E000FF00FF00FF00FF00FF00FF00FF00FF00D6
:1042F000FF00FF00FF00FF00FF00FF00FF00DD00E8
:00000001FF
